:020000040800F2
:10000000008000300D2300082D1700082D17000870
:100010002D1700082D1700082D17000800000000FC
:100020000000000000000000000000002F17000882
:100030002F170008000000002F170008DD1A000825
:100040002D1700082D1700082D1700082D17000880
:100050002D1700082D1700082D1700082D17000870
:100060002D1700082D1700082D170008ED1A00089D
:100070002D1700082D1700082D1700082D17000850
:100080002D1700082D1700082D1700082D17000840
:100090002D1700082D1700082D1700082D17000830
:1000A0002D1700082D1700082D1700082D17000820
:1000B0002D1700082D1700082D1700082D17000810
:1000C0002D1700082D1700082D1700082D17000800
:1000D0002D1700082D1700082D1700082D170008F0
:1000E0002D1700082D170008000000002D1700082C
:1000F0002D1700082D1700082D1700082D170008D0
:100100002D1700082D1700082D1700082D170008BF
:100110002D1700082D1700082D1700082D170008AF
:100120002D1700082D1700082D1700082D1700089F
:100130002D1700082D1700082D1700082D1700088F
:1001400000000000000000000000000000000000AF
:100150002D1700082D1700082D1700082D1700086F
:100160002D1700082D1700082D1700082D1700085F
:100170002D1700082D1700082D170008000000009B
:100180002D1700082D1700082D1700082D1700083F
:10019000311700082D1700082D1700082D1700082B
:1001A0002D1700082D1700082D170008000000006B
:1001B0002D1700082D1700082D1700082D1700080F
:1001C0002D1700082D170008000000000000000097
:1001D00000000000000000002D17000800000000D3
:1001E000000000000000000000000000000000000F
:1001F00000000000000000002D1700082D17000867
:100200002D1700082D170008000000002D1700080A
:100210002D1700082D1700082D1700082D170008AE
:100220002D170008000000002D1700080000000036
:100230002D1700082D170008000000002D170008DA
:100240002D1700082D1700082D1700082D1700087E
:100250002D1700082D1700082D1700082D1700086E
:100260002D1700082D1700082D1700082D1700085E
:100270002D1700082D1700082D170008000000009A
:100280002D1700082D1700082D1700082D1700083E
:10029000000000002D1700082D17000800000000C6
:1002A000000000002D1700082D1700082D1700086A
:1002B0002D1700082D1700082D1700082D1700080E
:0C02C0002D1700082D1700082D1700084E
:1002CC0044F20041C5F602010869C0F3C2000328DC
:1002DC0014D002280DD090BB0868800649F20000AB
:1002EC00C0F2D03058BF70470968C1F3C101C84093
:1002FC00704747F64000C0F27D1070478A6A886AE2
:10030C00C0F3051CC86ABCF1000F4B6B04BF002086
:10031C00704700F0010002F003024042022A00EA9A
:10032C00D3006FF35F3000EE100AB8EE400A0BD02A
:10033C006AB9086880060DD49FED221A17E040F6C2
:10034C000010C0F23D0070479FED1D1A0FE09FEDAD
:10035C001B1A0CE0086849F20002C0F2D032C0F35C
:10036C00C10022FA00F001EE100AB8EE411A086B37
:10037C009FED153A6FF35F2002EE100A086BC0F385
:10038C004620B8EE422A013000EE032A00EE10CAD5
:10039C00B7EE003AB8EE400A81EE000A32EE031ACC
:1003AC0020EE010A01EE100AB8EE411A80EE010AA5
:1003BC00BCEEC00A10EE100A704700BF0024744A4D
:0C03CC0020BCBE4B0024744C0000003923
:1003D8002DE9F8430446C07844F210460007C5F6F4
:1003E800020621D5606E4FEA3051032931D8DFE883
:1003F80001F002070D16F16941F40031F1610EE0D8
:1004080004F10800022101F08DFD04E004F1280048
:10041800022101F00FFE5FEA000807D1606E316C1F
:1004280021F44011084330644FF000086078C00799
:1004380001D1454624E0A06D042835D84546DFE8BB
:1004480000F003110B171700F06940F40030F06159
:100458000EE04FF00108E9E704F12800002101F05F
:10046800E9FD04E004F10800002101F05BFD054608
:100478002F4635B9306CA16D20F007000843306471
:100488004746607840072AD5D4F8A4004FEA705050
:10049800052812D8DFE800F003140B1A1A1AF069BD
:1004A80040F40030F06111E001250127E9E704F18B
:1004B8002800002101F0BEFD07E00125A8460FE055
:1004C80004F10800002101F02DFD0546A8463DB9BC
:1004D800B06CD4F8A41020F460000843B064B846A7
:1004E8006078000727D5D4F8A8004FEA30600528BF
:1004F8000FD8DFE800F0031108171717F06940F468
:100508000030F0610EE004F12800002101F092FDB6
:1005180007E0012501270FE004F10800002101F0A0
:1005280001FD05462F463DB9B06CD4F8A81020F05F
:10053800E0600843B0644746E07880071BD5E06C6C
:100548004FEA3010032829D8DFE800F00D02070D24
:10055800F06940F40030F06105E004F10800022180
:1005680001F0E0FC0546A84635B9F06BE16C20F0D7
:1005780030000843F063B8466078C00625D5E06DC2
:100588004FEA3030042835D8DFE800F003110B17A4
:100598001700F06940F40030F0610EE00125A8462C
:1005A800EAE704F12800002101F044FD04E004F129
:1005B8000800002101F0B6FC05462F4635B9306C1D
:1005C800E16D20F4E04008433064474660788006D7
:1005D80021D5206E4FEA3040052800F2FB82DFE883
:1005E80000F012030C12121204F10800012101F0AC
:1005F80099FC07E001250127E8E704F1280001211B
:1006080001F018FD0546A84635B9306C216E20F476
:10061800E02008433064B8466078400620D5D4F816
:10062800AC004FEA3070052800F2D782DFE800F00E
:100638000F03090F0F0F04F10800012101F072FCEC
:1006480004E004F12800012101F0F4FC05462F46DE
:100658003DB9B06CD4F8AC1020F0E0400843B06469
:100668004746607800061AD5E06E80B1B0F1005FA9
:1006780007D0B0F1805F22D1F06940F40030F0611A
:1006880005E004F10800012101F04CFC0546A846EC
:1006980035B9306CE16E20F0405008433064B846FC
:1006A800E078C0071CD0A06C03284BD8DFE800F026
:1006B80010020A10F06940F40030F06108E00125EA
:1006C800A846EDE704F10800022101F02BFC0546DD
:1006D800294635B9F06BA16C20F003000843F0639C
:1006E8004146D4E90002420201D4884617E0D6F810
:1006F800F02342F48072C6F8F02340F22412C3F2C9
:1007080000021368D6F8F073FF0506D41768FF1ABD
:10071800642FF7D90325A84601E0A846ADB1C00764
:1007280062D0A06F4FEAF000052800F25982DFE896
:1007380000F053034D53535304F10800012101F015
:10074800F1FB48E001250121CBE7336ED4F8B0C0B6
:1007580083EA0C0313F4407F0BD0336E376E47F4F3
:1007680080373766376E23F4407327F4803737664F
:100778003366BCF5807F11D1176841F288330325B1
:10078800D6F860805FEA887808D4D2F80080A8EBB1
:10079800070898454FF00308F2D9C0E733684FF6C9
:1007A800CF770CF4407223F47C53C0F2FF0707EABA
:1007B8001C170025B2F5407F08BF3B4333606FF339
:1007C8001F3C326E42EA0C0232668EE704F12800C2
:1007D800012101F02FFC05462F4635B9706CA16F39
:1007E80020F03800084370644746207880071CD5FD
:1007F800606F052800F2F781DFE800F00F03090FAA
:100808000F0F04F10800012101F08CFB04E004F152
:100818002800012101F00EFC0546A84635B9706C88
:10082800616F20F0070008437064B84620784007DD
:100838001ED5D4F89000052800F2D881DFE800F032
:100848000F03090F0F0F04F10800012101F06AFBE3
:1008580004E004F12800012101F0ECFB0546A9465B
:100868003DB9B06CD4F8901020F007000843B0648C
:10087800C1462078800620D5D4F88C004FEA307025
:10088800052800F2B681DFE800F00F03090F0F0F0B
:1008980004F10800002101F045FB04E004F1280000
:1008A800022101F0C7FB05462F463DB9706CD4F80C
:1008B8008C1020F0E040084370644F4620784006D2
:1008C80020D5D4F898004FEAB020052800F294818A
:1008D800DFE800F00F03090F0F0F04F108000021F3
:1008E80001F020FB04E004F12800022101F0A2FB42
:1008F8000546A8463DB9B06CD4F8981020F4E050ED
:100908000843B064B8462078000620D5D4F89C0087
:100918004FEA7030052800F27281DFE800F00F031B
:10092800090F0F0F04F10800002101F0FBFA04E0A1
:1009380004F12800022101F07DFB05462F463DB950
:10094800B06CD4F89C1020F460400843B06447466B
:10095800D4E90001010715D5D4F88000B0F5805F0F
:1009680009D104F12800022101F064FB002818BF16
:100978000127D4F88000716C21F440510843706459
:10098800D4E90001C10615D5D4F89400B0F5807FEC
:1009980009D104F12800022101F04CFB002818BFFE
:1009A8000127D4F89400B16C21F440710843B06475
:1009B800D4E9000100031FD5D4F8A000B0F5003F2A
:1009C80011D0B0F5803F08D0002840F0FB8004F13A
:1009D8000800002101F0A6FA04E004F12800022131
:1009E80001F028FB0546A8463DB9B06CD4F8A01024
:1009F80020F440300843B064B846A07840071FD5BB
:100A0800D4F88400B0F5401F11D0B0F5001F08D00D
:100A1800B0F5801F40F0D980F06940F40030F061F3
:100A280005E004F12800012101F004FB05462F46EA
:100A38003DB9706CD4F8841020F4401008437064F9
:100A48004746A078C00701D1B8461AE0206DB0F536
:100A5800803F05D098B9F06940F40030F06105E0B6
:100A680004F10800022101F05DFA0546A84645B9DF
:100A7800F06B216D20F480300843F063E4E7012532
:100A8800A846D4E900108A000AD504F128000221FA
:100A980001F0D0FA002818BF4FF00108D4E900107F
:100AA8008A0316D5E26F6FF0010303EB3223022BA2
:100AB80009D34FEA322333B1012B40F08980F3691F
:100AC80043F40033F3612DB9736C23F440731A4374
:100AD80072644546CA0205D5326C236F22F0004283
:100AE8001A4332648A0205D5326CA36E22F08072F2
:100AF8001A4332644A0008D5326822F40042326050
:100B0800D4F8B42033681A433260CA0F05D0F26BA8
:100B1800636D22F040521A43F263090206D5716CE4
:100B2800D4F8882021F4400111437164C10709D029
:100B380004F10800002101F0F5F9002818BF054666
:100B4800D4E90010810709D504F10800012101F05A
:100B5800E9F9002818BF0546D4E90010410709D56E
:100B680004F10800022101F0DDF9002818BF05464C
:100B7800D4E90010010709D504F12800002101F08B
:100B880059FA002818BF0546D4E90010C10609D54E
:100B980004F12800012101F04DFA002818BF05468C
:100BA800D4E90010800607D504F12800022101F0DD
:100BB80041FA002818BF0125002D18BF0125284635
:100BC800BDE8F8830125A84617E70125012738E77E
:100BD80001257FE70125A8461EE50125012740E5F7
:100BE8000125012701E60125A8461FE60125A9469A
:100BF8003FE60125012761E60125A84683E6012590
:040C08000127A5E635
:100C0C00034C206804348047FBE700F07AFAFEE7D7
:040C1C003423000875
:100C200000220B0011001A0084465AB3830704D037
:100C300000F8011B013AF9D124E0C9B241EA0121CF
:100C400041EA0141202A11D3203A2DE9F0030B4655
:100C50000C460D460E460F4688468946A0E8FA0324
:100C6000203AFBD2BDE8F00320320BD0042A05D392
:100C700040F8041B043A05D0042AF9D200F8011BFD
:080C8000013AFBD16046704708
:100C88002DE9F04FB1B040F2000443F60001C3F281
:100C980000040020C4F200012768A06201F5784032
:100CA8008F42A0F5744504D0AF4218BF874240F088
:100CB800D580E26B0126E368083306EB5212DB08A5
:100CC8008F4203FB02F218BF874240F0BB80102A14
:100CD80000F2C88094F88100002840F081810CA8B7
:100CE8009021002684F88060FFF796FF05F578408C
:100CF800874240F075814FF400500221CDE9020689
:100D08000320049028200B96CDE905010B20CDE99E
:100D18000701C020CDE909064FF480301A9002A8D7
:100D2800FFF756FB002840F0ED8144F2E04141F224
:100D3800000CC5F60201C5F6020C4FF0010A4FF08F
:100D48000F0E08694FF0050B40F400500861086960
:100D5800002300F4005001900198086840F010004A
:100D68000860096801F010010191019900210AFA4F
:100D780003F919F4B04F2BD00320DCF8088000FAEF
:100D880001F7C04328EA0705CCF80850DCF80450FE
:100D980025EA0909CCF80490DCF80C9000EA530520
:100DA80029EA07096544CCF80C9006F01C092A6A60
:100DB8000EFA09F022EA00000BFA09F21043286241
:100DC800DCF800000222B8438A401043CCF8000047
:100DD8000133043602310F2BC9D140F28800542167
:100DE800C3F20000002740F2241208254160402188
:100DF800C0E902174FF4806101614FF4006141615D
:100E08004FF40051C3F20002C4F202050226C0E901
:100E18000617C0E908772946136880F8356051F845
:100E2800086F016080F8347026F001070F60A96828
:100E3800C90719D01168C91A0529F8D94FF0030E46
:100E480020266AE0AF4218BF082A0BD805F574407F
:100E5800874218BFAF423FF43AAF3BE7E2680F2A38
:100E68007FF627AF01203DE148F23F02A968CFF69F
:100E780010620A40D0E903391A43D0E9051E42EA54
:100E88000902D0F82490D0E9076311433143D0E92F
:100E98000BA71943B9F1040F47EA0A02D0E9018CFC
:100EA80008BF1143A8F13F0241EA0C01132A41EAA5
:100EB8000E0307D80121914040F20F32C0F20F0211
:100EC800114204D1A8F12901062980F00E8143F4CA
:100ED8008013AB60B9F1040FE96921F0070149EA11
:100EE80001092CD1836ABAF1000F49EA030926D017
:100EF800BEF5005F08D0BEF1000F18D1022B19D043
:100F0800012B0ED0B3B11AE0032B18D84FF0010E05
:100F18004026DFE803F0020F0206466580F835E058
:100F280072B6AAF1C071B1FA81F14B0904E0032B42
:100F380040F0E280CAF30063002B40F0DF8040F607
:100F48008007C4F202070021C4F20201C5F81C9010
:100F58000023C0E916133F210126BCF1800F296048
:100F680005F5FF61C0E91817866604D14360C5F826
:100F7800F8377E6016E0A8F101015FFA88F30729C7
:100F8800C5F8F8377E600DD8013B082B0FD207EB68
:100F9800880107F1C0027C3106FA03F3C0E91B128D
:100FA800436707E000214167C0E91B1105E000F134
:100FB8006C010EC900270F6053600021416580F85D
:100FC8003560A06784634EF60C50CEF20000A0F6A0
:100FD8000442006882F84C134FF4801010602768B0
:100FE800022084F88100386820F001003860B86871
:100FF800D4F81880B8F1806F00F4F81ED4F804A073
:1010080010D1BAF1000F05D0BAF5800F0AD1A36B41
:1010180073B903E0A36BB3F1805F06D13B6843F477
:1010280080533B605FEA4A2302D44FF0010C0BE087
:10103800E6684FF0000C072E06D33B68256D23F4B5
:1010480080732B433B6004E03E6826F480763E6064
:10105800E668E26946EA0E06A16A3243E66B114386
:10106800D4F808B03143D4E90493B960D4E90D1534
:10107800626A1143226A294341EA09011943D4E902
:1010880012061143A26D314341EA0B010843104394
:10109800BAF1000F40EA080040EA0A00F8600DD0F3
:1010A800386DBCF1000F20F00100386514D1F868E4
:1010B800616D20F000400843F8600DE0B868012138
:1010C80061F3CC20B860B868022161F34A20B860A7
:1010D800386D20F0010038650020C4F88400012133
:1010E80084F8811031B0BDE8F08F28F0030174292D
:1010F80008BF43F48013ECE6BFF421AF4FF0010EB4
:0611080040260AE772B662
:10110E00AEB04EF60C54BFF35F8FCEF20004A06962
:10111E0020F48030A0610020C4F88800C4F88C0050
:10112E00D4F8941021F00101C4F8941048F23F71E4
:10113E00C4F89000C1F20401C4F894100521C4F85B
:10114E008810A16941F48031A161BFF34F8FBFF3C5
:10115E006F8FA168890311D4BFF34F8FBFF36F8FC9
:10116E00C4F84402BFF34F8FBFF36F8FA06840F4F3
:10117E000030A060BFF34F8FBFF36F8FA068C00326
:10118E0025D40020A067BFF34F8F43F6E077616F41
:10119E00C1F34E30C1F3C902C908551C430103EA1D
:1011AE00070202EB81762A46013AC4F8546206F130
:1011BE004046F9D1203B0138F1D2BFF34F8FA068E2
:1011CE0040F48030A060BFF34F8FBFF36F8F206865
:1011DE004FF6FF01084040F2003144F20045C0F2E4
:1011EE00FA51C5F6020508432060FFF768F8A969B1
:1011FE0042F22437C0F6000740F22C18C1F3032147
:10120E00C3F20008795C01F01F01C840A969C8F853
:10121E0000000F2000F013FC58B9D5F8F40040F090
:10122E000200C5F8F400D5F8F40000F002000090BA
:10123E00009805F20C4040F22416C3F20006016835
:10124E00490701680DD5022262F30201016031687F
:10125E0050F8082C920404D43268521AB2F57A7FF0
:10126E00F6D900210091C168022262F38F31C1606C
:10127E00C16801F4404100910099C1688904FCD510
:10128E00D5F8000440F48070C5F80004286F20F0F3
:10129E0018002867286900F03801A86A102907D0BD
:1012AE00182940F06C8100F00300022840F067819D
:1012BE002868D5F8000440F48070C5F80004306842
:1012CE00D5F80014C90504D43168091A6429F7D970
:1012DE00AAE1286F41F2883140F00100286730689A
:1012EE002A6F920704D43268121A8A42F8D99BE107
:1012FE00286900F03800182840F04F81A86A40F2A3
:10130E00F33108405228286B40F08E8101466FF36E
:10131E005F21272940F0888100F47E41B1F5007FDE
:10132E0040F0828100F4FE01B1F5803F40F07C81F7
:10133E0000F0FE40B0F1807F40F07681686B4FF692
:10134E00F871084210D0E86A20F00100E8623068B7
:10135E0031688142FCD0686B4FF6F8718843686340
:10136E00E86A40F00100E86242F20000C5F2002097
:10137E00016809070AD10168012262F303010160C5
:10138E00016801F00F01012940F0C781A969E969DF
:10139E00E969296AA969A96921F47061A9612968B5
:1013AE00890140F1BA812969032262F302012961A0
:1013BE00316841F288322B6903F03803182B04D0C0
:1013CE0033685B1A9342F6D9A7E1A969090703D0DE
:1013DE00A96921F00F01A961016811F00E0F0AD061
:1013EE000168012262F303010160006800F00F0042
:1013FE00012840F09281A86910F0700F03D0A869FF
:10140E0020F07000A861E86910F0700F03D0E86951
:10141E0020F07000E861E86910F4E06F03D0E8692D
:10142E0020F4E060E861286A10F0700F03D0286A9B
:10143E0020F070002862FEF742FFA96940F22812E0
:10144E00C3F20002C1F30321795CAB69127801F09B
:10145E001F0120FA01F11020002AC8F8001018BF51
:10146E000F2000F0ECFA002840F05781D5F8E0008C
:10147E0040F2041740F00400C5F8E000D5F8E00093
:10148E0044F2080800F00400009000984FF4006148
:10149E00D5F8E000C3F2000740F08000C5F8E00088
:1014AE00D5F8E000C5F6000800F080000090009826
:1014BE00D5F8E00040F01000C5F8E000D5F8E000E7
:1014CE0000F0100000900098D5F8D80040F0010010
:1014DE00C5F8D800D5F8D80000F0010000900098AB
:1014EE0020684EF20B400024CEF2000004704EF243
:1014FE000010CEF2000001607F21A8F1080047E93C
:10150E0001047960FF21C7E90214C7E90444BC61F4
:10151E00797FB9B902A8B0213C77FFF77AFB4FF477
:10152E008000CDE900044FF480702C906846FEF7E1
:10153E004CFF002840F0F280286F40F400402867EE
:10154E0057F8040C02217977C168C90600F1B880FA
:10155E00CA21416253214162C168490665D44FF0E8
:10156E00FF31C1603168C26852065ED43268521AC9
:10157E00B2F57A7FF7D903217977C06887E02868BA
:10158E0040F4803028603068296889033FF591AEB9
:10159E003168091A6429F7D946E0286820F080706E
:1015AE00286030682968890104D53168091A022932
:1015BE00F8D939E0A86A40F2F33188434FF6F87152
:1015CE005230A86240F22720C0F201102863E86A68
:1015DE0020F00100E862686B88436863E86A0221C4
:1015EE0061F38300E862E86A20F00200E862E86ACC
:1015FE0040F48030E862E86A40F40030E862E86A5D
:10160E0040F48020E862E86A40F00100E862286851
:10161E0040F0807028603068296889013FF5A4AEDB
:10162E003168091A0229F7D972B6816821F4E001EE
:10163E0021F04001816097E84E0031437E693143CD
:10164E0086683143816043EA02410161D8F80400A3
:10165E0020F08000C8F80400D8F80000800605D4F9
:10166E0000F01AFAF0B10320787710E0D8F80000F5
:10167E0020F02000C8F8000000F00EFA60B1032040
:10168E007877D8F8000040F02000C8F8000057F82E
:10169E00040CFF21416272B6D8F8000040F0200021
:1016AE00C8F8000057F8040C3969BA69C36C1143C5
:1016BE0023F00303C364C26C1143C164FF21416272
:1016CE00012040F21C047877C3F2000443F200407C
:1016DE001421C4F2010044F81C0C4FF4800044F8AD
:1016EE00180C4FF4C02044F8140C082044F8100CC9
:1016FE00002044E903004FF0005044F8040C20464B
:10170E00FFF787FA4FF08040A06104F11C002421FE
:0E171E00FFF77FFAFFF7B1FA72B672B672B635
:02172C00FEE7D6
:02172E00704702
:1017300038B540F20004C3F200042068026943692E
:10174000816894F881501D0507D512F008051FBF68
:10175000816941F40061816138BD03EA020505F049
:101760006402042A04D1616F20468847216F10E08B
:1017700005F04502012A07D1216F2046884705F070
:101780002200022804D038BD05F02602022A04D126
:10179000616F2046BDE8384008472A076BD415F42E
:1017A000587FF0D06A0609D5D4F8842042F00402AC
:1017B000C4F88420826942F040028261AA0509D5FA
:1017C000D4F8842042F00102C4F88420826942F4F3
:1017D00000728261EA0509D5D4F8842042F008023B
:1017E000C4F88420826942F480728261AA0609D515
:1017F000D4F8842042F08002C4F88420826942F048
:1018000020028261D4F88420002ABCD0026801F44E
:10181000404122F001020260026940F26B33B1F5EF
:10182000404F22EA0301016140F0B980816842F231
:10183000F92521F440418160E06FC0F6000550B108
:10184000056500F083FC00281EBFD4F8840040F03A
:101850004000C4F88400A06F002894D0056500F013
:1018600075FC002808BF38BDD4F8840040F0400063
:10187000C4F8840038BD816941F008018161816943
:1018800041F010018161816941F400618161016968
:1018900021F008010161816811F4404F24D1B4F8AE
:1018A0006A1009B3E168102905D32268616E126BD2
:1018B00041F8042B0DE0082904D3028E616E21F853
:1018C000022B06E0216891F83010626E1170616E93
:1018D00001316166B4F86A100139A4F86A10B4F8ED
:1018E0006A100029DED120684169826942F008024D
:1018F0008261826940F26F3342F0100282610268B5
:1019000022F00102026002699A430261826822F4B5
:101910004042826094F88120042A18BF11F020020E
:1019200009D0D4F8842042F08002C4F8842082696F
:1019300042F02002826194F88120032A18BF11F03E
:10194000400209D0D4F8842042F00402C4F8842074
:10195000826942F0400282618A0509D5D4F8842068
:1019600042F00102C4F88420826942F4007282616C
:10197000C90509D5D4F8841041F00801C4F88410D1
:10198000816941F4807181610020A4F86200A4F8AB
:101990006A00012084F88100D4F8840038BD012059
:0619A00084F8810038BD4F
:1019A6004EF6885042F20003CEF20000C5F2002344
:1019B600026842F470020260186800F00F00062800
:1019C60004D81868072262F30300186044F2004046
:1019D6004EF67F51C5F60200CEF6F621026842F0B9
:1019E6000102026000220261D0F800C001EA0C0187
:1019F60001601968090705D519684FF0070C6CF3E3
:101A06000301196040F200218261C0F20221C26125
:101A1600026281620021C0F2FF11C16240F28021A0
:101A2600C0F20111016342638163C26301644264CF
:101A3600016821F480210160026603F5005043F23B
:061A4600D20101607047AF
:101A4C0010B540F22C1144F6D352C3F20001C1F28E
:101A5C00620201240968A1FB0212A11E01EB921182
:101A6C000A0E18D14EF21002F023CEF20002516091
:101A7C0002F613510B700021916007210F281160A1
:101A8C0009D8A01E0F2100F025FA40F22810C3F24D
:0A1A9C00000004700024204610BD75
:101AA60040F200104FF65F71C3F20000C0F203016E
:101AB6000068C16040F22411C3F200010A68C368DD
:101AC6009B0606D40B689B1AB3F57A7FF7D90320D9
:061AD6007047002070477C
:101ADC0040F22410C3F2000001680131016070472C
:101AEC002DE9F04782B00020019040F22C1040F21A
:101AFC008804C3F20000C3F2000448F2B51240F2AD
:101B0C006F480168C1F64E32A56DC4F20208206818
:101B1C00A1FB021A40452F68296808DCA8F57471EE
:101B2C00884211DC4839884225DC473924E045F2EB
:101B3C002F42C5F60202904214DC08F14802904292
:101B4C003BDCA2F1470117E001F56271884212DC1F
:101B5C00A1F28731884218D01831884215D001F58E
:101B6C0056710FE03C329042D4BF3B3A0132904266
:101B7C0030D0143228E00131884206D01831884226
:101B8C0003D01831884240F09881E16D082201F0B1
:101B9C001F01A8F160098A403A4267D004234845E6
:101BAC0006DCA8F58066B042D4BF303E303647E044
:101BBC00404543DCA8F1300642E001329042E4D0CB
:101BCC0045F20842C5F60202904203D0143290420C
:101BDC0040F073810268E36D03F01F0304279F40FC
:101BEC000F4218BF12F004061CD102279F400F426F
:101BFC0018BF12F0020640F0B780D940090740F137
:101C0C005C8112F0080100F05881016821F00E018E
:101C1C000160012000FA03F16960606584F8350009
:101C2C00E16C00E111046F6000F1B080910600F1ED
:101C3C00B180016821F004010160ABE008F13006CD
:101C4C00B042CCBF01362F3EB04203D01836B04262
:101C5C0018BF082306681E4208D0036823F004034B
:101C6C000360AA60626D42F00102626501228A4043
:101C7C003A4221D0484506DCA8F580639842D4BF8F
:101C8C00303B303306E0404502DCA8F1300301E084
:101C9C0008F130039842D4BF2F3B0133984203D054
:101CAC001833984240F0128143691B0604D5AA6090
:101CBC00626D42F00202626504228A403A4221D0EF
:101CCC00484506DCA8F580639842D4BF303B3033DE
:101CDC0006E0404502DCA8F1300301E008F13003D6
:101CEC009842D4BF2F3B0133984203D0183398420B
:101CFC0040F0EE8003689B0704D5AA60626D42F049
:101D0C000402626510228A403A424CD008234845AE
:101D1C0006DCA8F58066B042D4BF303E303606E013
:101D2C00404502DCA8F1300601E008F13006B04273
:101D3C00CCBF01362F3EB04203D01836B04218BF8C
:101D4C00042306681E422ED0AA6002685203026861
:101D5C0006D4D20506D4026822F00802026001E023
:101D6C00100319D4226C18E011046F6000F1A880E4
:101D7C00910600F1A980016821F00A01016001209F
:101D8C0084F83500002084F834009DE0D00301D4A1
:101D9C00A16C89E0216C87E0A26C22B120469047AF
:101DAC00E06D00F01F01202000FA01F23A425AD0F7
:101DBC0020681023484506DCA8F58067B842D4BFDC
:101DCC00303F303706E0404502DCA8F1300701E037
:101DDC0008F13007B842CCBF01372F3FB84203D0CF
:101DEC001837B84218BF022307681F423BD0AA60BD
:101DFC0094F83520042A02681AD122F016020260E7
:101E0C00426922F080024261226CA36C1A4303D017
:101E1C00026822F0080202603F208840A86001207E
:101E2C0084F83500216D002084F83400E9BB44E0CF
:101E3C00510301680CD4C9050ED4016821F01001BE
:101E4C000160012084F83500002084F8340003E0A0
:101E5C00080301D4616C00E0E16B21B140F2880011
:101E6C00C3F200008847606D38B3606DC0071AD0AC
:101E7C00042084F835002068016821F0010101601C
:101E8C00019901310191B1EB9A2F02D80168C90770
:101E9C00F6D10068C00714BF0320012084F8350078
:101EAC00002084F83400E16C39B140F28800C3F2B0
:101EBC00000002B0BDE8F047084702B0BDE8F0876B
:101ECC00D00301D4616CEFE7E16BEDE70268F3E658
:041EDC00026817E79A
:101EE00000B54EF60C5C4FF0FF3ECEF2000CDCF875
:101EF0000030C3F3022383F00702042A28BF042220
:101F00000EFA02F29143033B00F00F0228BF994002
:101F100000F16043043A03F56443624400284FEA49
:0C1F2000011048BF02F10C03187000BD56
:101F2C0070B544F20043C5F60203D3F828E00EF076
:101F3C00030EBEF1030F04BF012070BD40F2241C40
:101F4C00D3F800E0C3F2000C2EF0806EC3F800E072
:101F5C00DCF800E01A68120106D5DCF80020A2EBD0
:101F6C000E02022AF6D95FE09A6A0129D0E900E450
:101F7C0022F47C32D0E9025642EA0E329A624FF4D5
:101F8C007E42A4F1010E02EB452204696FF35F2E31
:101F9C004FF0FE451EFA82F24FF4FE0E0EEB064E8B
:101FAC000EF4FE0E05EB0464724404F0FE4E724413
:101FBC009A63DA6AD0F814E022F0C00242EA0E0208
:101FCC00DA62DA6AD0F818E022F0200242EA0E0255
:101FDC00DA62DA6A4FF6F87E22F01002DA62DA6B15
:101FEC00C06922EA0E0242EAC000D863D86A40F007
:101FFC001000D8624FF4001008BF4FF48010002975
:10200C00D96A08BF4FF400200843D862186840F022
:10201C0080601860DCF800001968090106D4DCF84F
:10202C000010091A0329F7D3032070BD002070BDDE
:10203C0070B544F20043C5F60203D3F828E00EF065
:10204C00030EBEF1030F04BF012070BD40F2241C2F
:10205C00D3F800E0C3F2000C2EF0805EC3F800E071
:10206C00DCF800E01A68920006D5DCF80020A2EB40
:10207C000E02022AF6D95FE09A6A0129D0E900E43F
:10208C0022F07C72D0E9025642EA0E529A624FF468
:10209C007E42A4F1010E02EB452204696FF35F2E20
:1020AC004FF0FE451EFA82F24FF4FE0E0EEB064E7A
:1020BC000EF4FE0E05EB0464724404F0FE4E724402
:1020CC001A64DA6AD0F814E022F4406242EA0E0292
:1020DC00DA62DA6AD0F818E022F4007242EA0E02F0
:1020EC00DA62DA6A4FF6F87E22F48072DA625A6C9F
:1020FC00C06922EA0E0242EAC0005864D86A40F471
:10210C008070D8624FF0807008BF4FF40000002937
:10211C00D96A08BF4FF480000843D862186840F0B1
:10212C0080501860DCF800001968890006D4DCF8CF
:10213C000010091A0329F7D3032070BD002070BDCD
:10214C0090F83510022916D180B540F20F42016883
:10215C00C4F20202914212DCA2F5687C61451DDCDE
:10216C00A2F5747C61452FDCA2F2FF3C614548D09E
:10217C00A2F2E73C43E080214165012163E002F1DA
:10218C00600C614515DC02F1300C614523DC02F179
:10219C00010C614535D002F1190C30E0A2F55C7CE4
:1021AC0061451FDCA2F29F3C61452AD0A2F2873C1C
:1021BC0025E002F1900C61451BDC02F1610C6145DC
:1021CC001FD002F1790C1AE0A2F2CF3C614518D075
:1021DC00A2F2B73C13E002F1310C614511D002F1CF
:1021EC00490C0CE0A2F26F3C61450AD0A2F2573CBC
:1021FC0005E002F1A90C614503D002F1910C614597
:10220C0028D191424FF0040280F8352006DC6F2073
:10221C00C4F20200814207DD303006E040F26F402C
:10222C00C4F20200814203DC3038814203DD03E05A
:10223C003030814209DC2F38086820F0010008603A
:10224C000021BDE80840084670471930814218BF8C
:10225C001838F1E70A6822F00E020A6045F257427C
:10226C00C5F6020291420A6822F001020A6007DCFC
:10227C0045F22F42C5F60202914207DD013206E01B
:10228C0045F27F42C5F60202914204DC273A9142A4
:10229C0007D0143203E01532914202D0143A914225
:1022AC0019D1D0E91813D0E916EC0A6822F480721F
:1022BC000A600CF01F01012202FA01F1CEF80410A1
:1022CC00816E5960C16E31B10A6822F480720A6065
:1022DC00D0E91C124A60012180F83510026D0021F2
:0C22EC00002A80F83410ACD09047A9E71D
:1022F800806B0021A0F86A10A0F86210012180F814
:042308008110704789
:10230C00FFF74BFB4EF68850CEF20000016851F4FB
:08231C0070010160FEF774FC82
:102324000000000000000000010203040607080981
:102334005923000800000030290100006B23000825
:102344002C0100305423000804000000170C00087E
:042354000090D00322
:10235800206861680834002200E042540139FCD545
:022368007047BC
:10236A0020686168A2680C3401E08B5C8354013AEE
:04237A00FBD57047D8
:040000050800230DBF
:00000001FF
